:100000009302000273A0023137010100FD28A948C4
:100010007300000082808548730000008280914850
:10002000730000008280AD48730000008280930856
:1000300010087300000082809308500873000000CD
:10004000828093087008730000008280732510C0BE
:100050008280732500C082809308600873000000CE
:1000600082800589F322008093920248B3E2A200C5
:10007000739002808280954873000000828093080C
:100080000008730000008280A14873000000828095
:1000900093083008730000008280930840087300C2
:1000A0000000828052B8BD450145D13F130440464F
:1000B00022950345A5006888BD450145C9372295AD
:1000C0000345A5002302A400BD4501454D3F2295EF
:1000D0000345A500A302A400BD4501454D37229567
:1000E0000345A5002303A400BD450145493F2295D2
:1000F0000345A500A303A400BD450145493722954A
:100100000345A5002304A40052BE46B822E44AE0F9
:100110000149130440461305100348889304340032
:10012000D149130519040888BD450145893F229529
:100130000345A5006888BD450145913722950345D3
:10014000A5002302A400BD450145153F22950345A6
:10015000A500A302A400BD4501451537229503451E
:10016000A5002303A400BD450145113F2295034589
:10017000A500A303A400BD45014511372295034501
:10018000A5002304A40066AC5D350509E31B39F91D
:100190000149130520034888D1491305190408882B
:1001A000BD450145E93D22950345A5006888BD454B
:1001B0000145F13522950345A5002302A400BD4564
:1001C0000145753D22950345A500A302A400BD4548
:1001D0000145753522950345A5002303A400BD45BF
:1001E0000145713D22950345A500A303A400BD452B
:1001F0000145713522950345A5002304A40066AC92
:100200003D350509E31B39F90149130530034888D9
:10021000D149130519040888BD4501458D3522953E
:100220000345A5006888BD450145913D22950345DC
:10023000A5002302A400BD45014591352295034543
:10024000A500A302A400BD450145153D2295034527
:10025000A5002303A400BD4501451535229503459E
:10026000A500A303A400BD450145113D229503450A
:10027000A5002304A40066AC5D3B0509E31B39F926
:100280000149130540034888D1491305190408881A
:10029000BD450145ED3322950345A5006888BD4560
:1002A0000145F13B22950345A5002302A400BD456D
:1002B0000145F13322950345A500A302A400BD45E5
:1002C0000145753B22950345A5002303A400BD45C8
:1002D0000145753322950345A500A303A400BD4540
:1002E0000145713B22950345A5002304A40066AC9B
:1002F0003D3B0509E31B39F90149130550034888C3
:10030000D149130519040888BD4501458D3B229547
:100310000345A5006888BD450145953322950345F1
:10032000A5002302A400BD450145913B229503454C
:10033000A500A302A400BD450145913322950345C4
:10034000A5002303A400BD450145153B22950345A7
:10035000A500A303A400BD4501451533229503451F
:10036000A5002304A40066ACD9310509E31B39F9C3
:100370000149130560034888D14913051904088809
:10038000BD450145ED3922950345A5006888BD4569
:100390000145F53122950345A5002302A400BD4582
:1003A0000145F13922950345A500A302A400BD45EE
:1003B0000145F13122950345A5002303A400BD4565
:1003C0000145753922950345A500A303A400BD4549
:1003D0000145753122950345A5002304A40066ACB0
:1003E000B9310509E31B39F91305100493054005DC
:1003F0007931088813051003930560034931488853
:10040000BD450145AD3922950345A5006888BD4528
:100410000145B53122950345A5002302A400BD4541
:100420000145B13922950345A500A302A400BD45AD
:100430000145B13122950345A5002303A400BD4524
:100440000145353922950345A500A303A400BD4508
:100450000145353122950345A5002304A40066AC6F
:04046000F93659B759
:1004640041310031323334353600303132333435B2
:0B04740036373839414243444546000A
:00000001FF
